:020000040800F2
:1000000000090020B10100083D310008F53000086A
:100010001D310008F530000815310008B301000853
:10002000B3010008B3010008B3010008B54100089E
:10003000B3010008B3010008B3010008B3010008D0
:10004000B3010008B3010008B3010008B3010008C0
:10005000B3010008B3010008B3010008B3010008B0
:10006000B3010008B3010008B3010008B3010008A0
:10007000B3010008B3010008B3010008B301000890
:10008000B3010008B3010008B3010008A93000085B
:10009000D5300008E5300008B3010008B3010008BE
:1000A000B3010008B3010008B3010008B301000860
:1000B00039550008B3010008B3010008B301000876
:1000C000B3010008B3010008B3010008B301000840
:1000D000B301000825550008B3010008B30100086A
:1000E000B3010008B3010008B3010008B301000820
:1000F000B3010008B3010008B3010008B301000810
:10010000B3010008B3010008B3010008B3010008FF
:10011000B3010008B3010008B3010008B3010008EF
:10012000B3010008B3010008B3010008B3010008DF
:10013000B3010008B3010008B3010008B3010008CF
:10014000B3010008B3010008B3010008B3010008BF
:10015000B3010008B3010008B3010008B3010008AF
:10016000B3010008B3010008B3010008B30100089F
:10017000B3010008B3010008B3010008B30100088F
:10018000B3010008B3010008B3010008B30100087F
:10019000B3010008B3010008B3010008B30100086F
:1001A000B91B0008FFFFFFFFFFFFFFFFFFFFFFFF7F
:1001B00002E000F000F8FEE772B6374880F30888E6
:1001C000364880F3098836483649086040F2000016
:1001D000CCF200004EF63471CEF200010860BFF39D
:1001E0004F8FBFF36F8F40F20000C0F2F0004EF669
:1001F0008851CEF200010860BFF34F8FBFF36F8FBD
:100200004FF00000E1EE100A4EF63C71CEF2000114
:100210000860062080F31488BFF36F8F04F096FF08
:1002200005F018F84FF055301F491B4A91423CBF6A
:1002300041F8040BFAE71D49184A91423CBF41F8C6
:10024000040BFAE71A491B4A1B4B9A423EBF51F86E
:10025000040B42F8040BF8E700201849184A9142B1
:100260003CBF41F8040BFAE704F074FF05F04AF8CC
:10027000144C154DAC4203DA54F8041B8847F9E7D7
:1002800000F0E8FB114C124DAC4203DA54F8041BA9
:100290008847F9E704F05CBF000900200011002046
:1002A0000000000808ED00E0000100200009002027
:1002B00098560008001100207811002078110020C5
:1002C000583E0020A0010008A4010008A401000875
:1002D000A40100082DE9F04F2DED108AC1F80CD0D3
:1002E000C3689D46BDEC108ABDE8F08F002383F300
:1002F00011882846A047002004F0B4FBFEE704F074
:1003000037FB00DFFEE7000080EA0102844612F0BE
:10031000030F4FD111F0030F32D14DF8044D11F0FE
:10032000040F51F8043B0BD0A3F101329A4312F0B1
:10033000803F04BF4CF8043B51F8043B16D100BF8A
:1003400051F8044BA3F101329A4312F0803FA4F11B
:1003500001320BD14CF8043BA24312F0803F04BFA2
:1003600051F8043B4CF8044BEAD023460CF8013B0F
:1003700013F0FF0F4FEA3323F8D15DF8044B7047B9
:1003800011F0010F06D011F8012B0CF8012B002AF7
:1003900008BF704711F0020FBFD031F8022B12F0E6
:1003A000FF0F16BF2CF8022B8CF8002012F47F4FA1
:1003B000B3D1704711F8012B0CF8012B002AF9D1A9
:1003C000704700BF10B4044C03460A4620685DF82D
:1003D000044B194604F0CCBD0011002010B5054CAB
:1003E00034B113460A4601460220AFF3008010BD27
:1003F000204610BD00000000024B0146186804F0C2
:10040000BBBD00BF00110020024B0146186804F07C
:10041000B7BD00BF0011002001292DE9F0415BD9D3
:100420004FF00108C64600244FF0FF35434608E070
:10043000A3EB05081C464FF0010E04EB0E03994296
:1004400010D900EB050CC75C1CF80E60B742EFD367
:1004500032D04FF001082546C646444404EB0E0353
:100460009942EED80127C2F80080BE4600244FF022
:10047000FF363B4607E09F1B1C464FF0010E04EB86
:100480000E03994210D900EB060C10F803801CF8FB
:100490000EC0E045EFD817D001272646BE463C44A3
:1004A00004EB0E039942EED80136681C864201D354
:1004B00017603046BDE8F081C6450ABF74440EF1AE
:1004C000010E4FF0010EB8E7BE450ABF74440EF1AD
:1004D000010E4FF0010ED2E701270026E8E700BF2A
:1004E0002DE9F04F164685B003AA0D46074619467A
:1004F00030461C46FFF790FFDDF80CA00246804610
:1005000006EB0A01304600F027FA2A1B002852D1D8
:1005100001468446A4EB0A0BC8F10109CDF804A0FA
:100520008845434638BF0B469C4219D95D1E03EBF4
:100530000C003544384402E001339C4210D010F8DE
:1005400001EB15F801AFF245F6D09C4208D9CC4436
:100550009C4400219445E3D9002005B0BDE8F08F0C
:10056000884508F1FF3367D908EB0C00384406EBE7
:100570000805CDF8008002E08B4212D0534615F8F2
:10058000018D10F801EDF04503F1FF3AF4D0DDF8EC
:10059000008001330131994208D8019B59469C449F
:1005A000D8E701319942DDF80080F6D907EB0C005D
:1005B00005B0BDE8F08FA4EB0801414538BF4146C6
:1005C000444501F101014FF0000C31D908F1FF3E23
:1005D000C8F101090CEB080006EB0E053844434650
:1005E00002E001339C4223D010F801AB15F801BFA3
:1005F000D345F6D09C421BD9CC449C449445ABD8FF
:100600004445E7D806EB08090CEB08053D4448468D
:1006100001E0B342CAD010F801AD15F801EDF24582
:100620000346F6D08C44944596D84445CED8EBE7A3
:10063000B8F1000FE6D1B9E74346ABE72DE9F04F3B
:100640001546ADF21C4D06468A4605AA19462846AF
:100650000093FFF7E1FE009B80460DF2144142F843
:10066000043F8A42FBD15C1E002B00F0CE80691E45
:1006700004EB050C06AF11F8010F5A1A013A2A448F
:10068000614547F82020F6D1DDF814B0009305EB62
:100690000B014246284600F05FF9009B0146AAEB99
:1006A000030A00285CD1A3EB0B03C8F101020093FD
:1006B000CDE901B20346A9460AE021B10199914270
:1006C000009988BF0A46134453454FF0000142D8B1
:1006D00006EB030C1CF8042057F82220002AECD16A
:1006E0008845424638BF0A46A24212D2551ED0184B
:1006F0004D44304402E00132A2420AD010F801EB2E
:1007000015F801BFF345F6D0A24202D202990B447C
:10071000D9E7884508F1FF327BD908EB0300304464
:1007200009EB0805CDF80C8002E08A426AD05A46EF
:1007300015F8018D10F801EDF04502F1FF3BF4D002
:10074000DDF80C8001320131914260D8019A0099A4
:1007500013445345BCD900200DF21C4DBDE8F08F69
:10076000A3EB080343454FF0000C38BF434606EBAC
:100770000C0001330193035D57F8233008F1FF3972
:10078000C8F1010B4BB19C44D445E4D806EB0C00F6
:10079000035D57F82330002BF5D1A04517D208EBA5
:1007A0000C02324405EB09014346CDF800C002E0DB
:1007B0000133A34223D012F801CB11F801EFE64533
:1007C000F6D0DDF800C0A34238BFDC44DBD3B8F17B
:1007D000000FC1D008EB0C01314405EB0802CDF845
:1007E00000C001E0AB42B7D012F801ED11F801CD25
:1007F000E6451346F6D0DDE900C39C44C4E7DDF8C6
:1008000000C0E4E7DDF80C809DE706AF3CE76046FA
:10081000A2E7424697E700BF2DE9F0470446C0B083
:10082000002B6AD0012B0D4690461F4600F08680B3
:100830008B425ED8CD1A022B00EB050661D0B3F5D2
:10084000807F00F282804FF48072002168465D1E36
:1008500001F0D4FA98F80010012240460B4610F837
:10086000011FA1EBC303DBB20DF803200132954257
:10087000F4D808EB07034FF0000A13F8022C18F81D
:100880000530A3EBC203DBB21DF803900DF8035053
:10089000A5EB0909B44201D92BE063B92C44A64267
:1008A00014F8013C94F800C0ACEBC30C5FFA8CFC6C
:1008B0001DF80C30F1D29D42A4EB0304EAD80F2DB1
:1008C00007D9042208EB0A0104EB0A0000F044F8FF
:1008D00060B92A464146204600F03EF868B1BAF1B8
:1008E000030F8CBFAAF1040AA7F1050A4C44B442D5
:1008F000D4D9002040B0BDE8F087204640B0BDE824
:10090000F08713785078217840EA0340234613F8A3
:10091000012F9E4242EA01421BD39042EDD00136A4
:1009200001E0904208D013F8011F9E4241EA0242C2
:10093000F7D18242DDD13346581EDBE711782A46D3
:1009400040B0BDE8F04700F035B840B0BDE8F04732
:1009500074E61E46EDE700BF032A30B415D941EA1C
:100960000004A40784460B4604D0541E0FE0043A4A
:10097000032A08D91946604653F8044B5CF8045B17
:10098000A542F4D0F1E760461946541E7AB1431EE1
:100990000139021901E09A4209D013F8010F11F848
:1009A00001CF6045F7D0A0EB0C0030BC70470020B1
:1009B00030BC704701F0FF01102A2BDB10F0070F4D
:1009C00008D010F8013B013A8B422DD010F0070FF0
:1009D00042B3F6D1F0B441EA012141EA014122F0EB
:1009E00007047FF000070023F0E80256083C85EA80
:1009F000010586EA010685FA47F5A3FA87F586FA26
:100A000047F6A5FA87F68EB9EED1F0BC01F0FF01EA
:100A100002F0070232B110F8013B013A83EA010308
:100A200013B1F8D10020704701387047002D06BF80
:100A300035460338073815F0010F07D1013015F49A
:100A4000807F02BF013015F4C03F0130F0BC013897
:100A5000704700BFF8B501F01BF904F015FB07461D
:100A600004F066FB0546A8BB1F4B9F4232D0013302
:100A70009F4232D01D4B27F0FF029A4230D1F8B28C
:100A800000F0F2FE2E4642F2107400F0F3FE08B1C0
:100A90000024264601F05EFC20B1032000F078F827
:100AA0000024264635B1124B9F4203D004F038FB98
:100AB00000242646002004F0F1FA0EB100F07EF882
:100AC00001F0F2F900F00AFF204600F0D3F800F040
:100AD00075F8F9E72E460024D7E704460126D4E747
:100AE00006464FF47A74D0E7010007B0000008B062
:100AF000263A09B008B501F099F8A0F12003584250
:100B0000584108BD07B5042101900DEB010001F02B
:100B1000A9F803B05DF804FB38B5302383F31188DE
:100B2000174803680BB104F05BF8164A1448002319
:100B30004FF47A7104F04AF8002383F31188124CC1
:100B4000236813B12368013B2360636813B16368B2
:100B5000013B63600D4D2B7833B963687BB902208C
:100B600001F036F9322363602B78032B07D16368D9
:100B70002BB9022001F02CF94FF47A73636038BD71
:100B800088120020190B00087C120020841200201B
:100B9000084B187003280CD8DFE800F0080502089D
:100BA000022001F00BB9022001F000B9024B002233
:100BB0005A607047841200207C12002010B501F0AA
:100BC000C9FB30B1244B03221A70244B00225A6017
:100BD00010BD234B234A1C4619680131F8D0043359
:100BE0009342F9D16268204B9A42F1D91F4B9B681E
:100BF00003F1006303F580339A42E9D204F062FA0C
:100C000004F074FA002001F05DF80220FFF7C0FF45
:100C1000174B9A6D00229A65996F9A67996FD96DF3
:100C2000DA65D96FDA67D96F196E1A66D3F8801052
:100C3000C3F88020D3F8803072B64FF0E023302123
:100C4000C3F8084DD4E9003281F311889D4683F33F
:100C500008881047BCE700BF841200207C120020E7
:100C60000000010820000108FFFF000850110020CB
:100C7000001002402DE9F04F93B0DFF8108301908F
:100C80002022FF210AA8D8F8086001F0B7F8B64A78
:100C90001378A3B9B548012103601170302383F3A1
:100CA000118803680BB103F09BFFB14AAF480023E2
:100CB0004FF47A7103F08AFF002383F31188019BBC
:100CC00013B1AC4B019A1A60AB4A019D1378032B08
:100CD0001EBF00231370A74A4FF0000A18BF5360CD
:100CE000D3465446D146012001F068F825B1A14B06
:100CF0001B68002B00F0F581002000F097FF071E15
:100D000038DB012001F052F8A7F121001628EAD8BB
:100D100001A353F820F000BF7B0D0008970D0008D9
:100D2000210E0008E70C0008E70C0008E70C00089B
:100D30009F0E0008551000084B0F0008D30F000845
:100D4000F90F00081F100008E70C00083110000818
:100D5000E70C00089D100008010E0008E70C0008D1
:100D6000E9100008870D0008010E0008E70C0008D4
:100D7000D30F000800F0F8FDB8E70220FFF7BAFE35
:100D8000002840F0E080019B7C48BAF1000F08BFCA
:100D90001D4602213EE04FF47A7000F047FF071E27
:100DA000F1DB0220FFF7A6FE0028ECD0013F052F63
:100DB00000F2C481DFE807F003070A0D10310520B7
:100DC000FFF7A0FE14E0D8F80000F9E7D8F8040017
:100DD000F6E7D8F80800F3E74FF01C09484600F0A2
:100DE00073FF09F10409FFF78DFEB9F12C0FF5D15E
:100DF0000123BB404BEA03035FFA83FB4FF000097A
:100E000001F048F824B10BF00B030B2B08BF0025B1
:100E10005B48022100F026FF65E7D8F80C00CFE719
:100E2000002CB0D00BF00B030B2B5AD10220FFF794
:100E300061FE0446002854D0012000F043FF022048
:100E4000FFF7A6FE00271FFA87FA504600F04AFF78
:100E5000054688B9484B012202201A7000F0A6FF0F
:100E60002E46D8F80830B34212D8434B00261E70E5
:100E7000404BA2465E60C3E70021504600F04AFFA7
:100E8000013705460028DED1A2463E480221C1E7CF
:100E9000304600F019FF0130F6D10436E1E7002CAE
:100EA0003FF471AF0BF00B030B2B1AD10220FFF7AD
:100EB0006FFE322000F0BAFE071E12DB17F00303AC
:100EC0000FD1D8F80810BA198A420AD8B7F5807F2E
:100ED00007D82D4A9F4206DCC820FFF70BFE0446C8
:100EE00080B901244FE74FF47A70CDE9023200F067
:100EF0009DFE0028FFF647AF039A029B02F8010B04
:100F00000133E7E71F2E11D8C6F12002BA420AAB1F
:100F100026F0030028BF3A461B490292184400F00D
:100F200061FF029A1848FF2100F068FFBB101649C4
:100F30000293C7F38702304600F068FF0028A4D070
:100F4000029B06EB830604465AE70220FFF7D2FD18
:100F500000283FF418AF00F0EFFE00283FF413AF75
:100F600000273B4627E000BF7812002088120020AF
:100F7000190B00087C1200208412002090550008F4
:100F8000945500088C55000878110020501100205D
:100F90001F2F18D80A9A013215D027F003024832C1
:100FA0006A4452F8200C05900422184605A901F065
:100FB000BBF904370346D8F80820BA42E8D81846E7
:100FC000FFF7A0FD1CE73846029300F07DFE029B70
:100FD000E9E70023642105A8059300F03BFE002803
:100FE0007FF4D1AE0220FFF785FD00283FF4CBAEA1
:100FF000059800F097FEE3E70023642105A8059318
:1010000000F028FE00287FF4BEAE0220FFF772FD3C
:1010100000283FF4B8AE059800F086FED0E7022025
:10102000FFF768FD00283FF4AEAE00F095FEC7E77D
:101030000220FFF75FFD00283FF4A5AE05A91420AC
:1010400000F090FE0746FFF75DFD394605A800F069
:1010500009FED5E6322000F0E9FD071EFFF693AE4B
:10106000BB077FF490AED8F8082007EB0903934242
:101070003FF689AE0220FFF73DFD00283FF483AE26
:1010800027F003074F44B9453FF4BAAE484600F095
:101090001BFEFFF737FD09F10409F4E74FF47A70FE
:1010A000FFF728FD00283FF46EAE00F045FE002853
:1010B0003FF4EBAE0A9B01330CD008220AA90020B2
:1010C00000F0A4FE00283FF4E0AE2022FF210AA891
:1010D00000F094FE1B48022100F0C4FD1A4803F002
:1010E000C7FC13B0BDE8F08F002C3FF44CAE0BF002
:1010F0000B030B2B7FF447AE0023642105A8059357
:1011000000F0A8FD074600287FF43DAE0220FFF75F
:10111000F1FC029000283FF436AE0221094800F0AD
:10112000A1FD41F2883003F0A3FC059800F0C8FE51
:1011300000F0B0FE029B3D461C46D4E54FF000098E
:1011400021E600BF94550008A0860100094A1368F3
:1011500049F2690099B21B0C00FB01331360064B86
:10116000186844F2506182B2000C01FB0200186062
:1011700080B27047641100206011002070B50C46E9
:1011800015461E4602F01EFB50B9022E10D1012D4D
:101190000ED112A3D3E90023C4E90023012007E004
:1011A000282D10D005D8012D09D0052D0FD00020F5
:1011B00070BD302DFBD10BA3D3E90023ECE70BA3CB
:1011C000D3E90023E8E70BA3D3E90023E4E70BA36B
:1011D000D3E90023E0E700BFAFF30080401DA1206A
:1011E00026812A0B78F6339F93CACD8D9E6AC4213F
:1011F000818A46EE26417272DF25D7B7F017304A52
:1012000039059E5610B500211022044600F0F6FD67
:10121000034B03CB206061601868A06010BD00BF65
:101220009075FF1FF0B5ADF5517D6EAC4FF4C472F3
:1012300007460D462046002100F0E0FD01F086FF44
:10124000264B4FF47A72B0FBF2F0186093E8070077
:10125000022384E807000DF5ED702382FFF7D2FF2B
:1012600048F604531E49238407A8FFF74DF81D23B1
:1012700084F832310DF2EB2207AB0DF1340C1E462F
:1012800003CE664510605160334602F10802F6D184
:1012900030681060337913710FAE31460122204659
:1012A00000F028FE80B2CDE9046000230393AB7EFA
:1012B000029305F11903019301230093E97E05A32D
:1012C000D3E90023384602F01FFB0DF5517DF0BD38
:1012D000AFF300809E6AC421818A46EEE0170020A9
:1012E000985500082DE9F0412C4C237ADAB080465D
:1012F0000D465BBB27A9284600F022FF07460028C1
:1013000042D19DF89D60C82E3ED801464FF4A6629A
:10131000204600F073FD4FF48073C4F8F8314FF4A9
:101320000073C4F80C3332464FF440730DF19E0144
:1013300004F10900C4F82034264400F053FD9DF860
:101340009C30777223720BB9EB7E237281220021CD
:1013500006AC27A800F052FD0122214627A800F084
:1013600035FF80B2CDE9044000230393AB7E0293A6
:1013700005F11903019328230093E97E05A3D3E91E
:101380000023404602F0C0FA5AB0BDE8F08100BF29
:10139000AFF3008026417272DF25D7B7A812002074
:1013A000F0B5254E4FF48A73F1B003FB00650024BD
:1013B00096F8D83085F8DC30D02221463CA885F854
:1013C000E84000F01BFD06F1090000F015FDD5F81E
:1013D000E4308DF8F000C2B206AF06F109010DF15C
:1013E000F100CDE93A3400F0FDFC394601223AA87B
:1013F00000F020FF80B2CDE9047008230127CDE979
:10140000023706F1D803019330230093317A0B4859
:1014100007A3D3E9002302F077FAA04206DD01F02A
:1014200095FEC5F8E000384671B0F0BD2046FBE7F8
:1014300078F6339F93CACD8DA8120020DC380020A7
:101440002DE9F0411D4D1E4E1E4F86B0284602F07C
:1014500087FA034658B30024CDE90344ADF814409D
:101460001A7B8DF8142058689968029403AA03C265
:101470001B68DFF8548043F00043029301F068FEDC
:10148000821941F10003009402A9384601F03EF9A7
:10149000A04205DD284602F067FA88F80040D5E74B
:1014A00098F80030072B05D8013388F8003006B0D3
:1014B000BDE8F081014802F057FAF8E7DC38002077
:1014C00040420F00F0170020A512002010B50021A7
:1014D000044600F01FFC601C0B4C80B2A4F82C05E5
:1014E00000F000FC70B1B4F82C0500F00BFC0146D4
:1014F00040B9B4F82C0500F00DFCB4F82C0501300F
:1015000080B2EBE710BD00BFA812002010B50A4B57
:101510000A4A1A6003F5805393F870203AB9DC6EDA
:101520002CB1204600F090FF204601F0CDF8BDE838
:101530001040034800F088BFF0170020FC55000859
:10154000482800202DE9F04F8FB000AF05460C462B
:1015500002F038F900284AD1237E022B1AD1E38AFF
:10156000012B17D101F0F2FD0646FFF7EFFD4FF416
:10157000C873DFF8EC82B0FBF3F206F5167602FBD7
:10158000130316FA83F3C8F80030E37E33B9AE4B89
:1015900000221A703C37BD46BDE8F08F07F12401E8
:1015A000204600F081FD0028F4D107F11400FFF778
:1015B00029FE97F8264007F11401224607F127007B
:1015C000FFF7CAF90028E2D10F2C08D89E4B1C70F7
:1015D000D8F80030A3F51673C8F80030DAE797F8AA
:1015E00024100029D6D0284602F0E4F8D2E7E38A96
:1015F000282B38D010D8012B30D0052BCAD1BFF3FF
:101600004F8F9249924BCA6802F4E0621343CB6059
:10161000BFF34F8F00BFFDE7302BBBD1DFF844B2E3
:10162000E17E9BF808209142B4D1607E59460022A9
:1016300091F8DC50854200F0B4800132042A01F5B3
:101640008A71F5D1DBF8002040F6B831FA328A42CF
:1016500094BFCBF80020CBF800109BE7214628462A
:10166000FFF7E0FD96E721462846FFF73BFE91E7AE
:10167000B2F8EC507B60EA1C930822F003020732B8
:10168000D208BB60A8EBC2039D46BB68EA469A003D
:101690000021504600F0B2FB7B6803F1EE012A46C0
:1016A0005944504600F09EFB14B9012000F00AFB9B
:1016B0009BF8D20000F016FB044638B98BF80800FE
:1016C00000F03AFB204600F0FDFAB4E0DBF8D4204D
:1016D0003AB99BF8D200BBF82C25824201D8FFF71B
:1016E000F5FEDBF8D4202A44944208D29BF8D200BD
:1016F000BBF82C250130824201D8FFF7E7FE3A7A89
:10170000DBF80400514600F081FB08B9C5467BE0D8
:10171000DBF804209BF8D2002A44CBF80420DBF845
:10172000D42005EB020ACBF8D4A000F0DBFA824506
:1017300009D39BF8D22001328BF8D220DBF8D420D9
:10174000121BCBF8D420FF2D10D800248BF80840B2
:1017500000F0F2FA204600F0B5FA00F0FBFD3D4B38
:10176000188108B9FFF72AFAC54613E7FB689BF80A
:10177000D90009FB03B2D2F8E41082F8E86001F561
:101780008061C2F8E060C2F8E410FFF709FEFFF7DD
:1017900057FE9BF8D920013202F003028BF8D920C2
:1017A000B4E74FF48A7909FB02F505F1EA015944DF
:1017B000204600F073FD064600287FF4EBAE5D4442
:1017C000012285F8E82001F0C1FCD5F8E020DBED2E
:1017D000007ADFED216A801A192838BF192040F6F7
:1017E000B832904228BF1046B8EE677A07EE900AEA
:1017F000F8EEE77A67EEA67ADFED186AE7EE267A6A
:10180000FCEEE77ACBED007A9BF8D930FB6009FB60
:1018100003F30BEB0302DBF8040092F8E81059B174
:10182000D2F8E4408442E8463FF422AF002182F837
:10183000E810C2F8E010C546DBF80430054A9B0A00
:1018400001331381A6E600BFD817002000ED00E0A9
:101850000400FA05E0170020CDCCCC3D6666663F5B
:10186000DC170020A8120020014B1870704700BF41
:10187000D828002038B54FF00054144B22689A4203
:1018800021D1607DF0B1124B124918701248237DAE
:1018900003724FF48073C0F8F8314FF40073C0F84E
:1018A0000C3300254FF44073C0F82034C0F8E450E6
:1018B000C922093000F096FAE0222946204600F0BD
:1018C0009DFA012038BD0020FCE700BF9AAD44C559
:1018D000D828002016000020A812002037B500F0FC
:1018E00039FD184D18492881022318486B7101F001
:1018F000D7FA00230193164B164900931648174B4D
:101900004FF4805201F02EFF154B197811B1124897
:1019100001F050FF01F01AFC0446FFF717FC4FF4EA
:10192000C87304F51674B0FBF3F202FB13000D4B01
:1019300014FA80F0186003F0FBFB08B10F232B8131
:1019400003B030BDE017002040420F00F017002028
:101950007D110008DC280020DC3800204515000837
:10196000D8280020DC1700202DE9F04F2DED028B48
:101970000FF23829D9E90089834C93B00BAD9FED64
:101980007E8BFFF75DFD814FDFF828A200230A93CD
:10199000ADF834300B936B604FF0000B5B468DED70
:1019A000008B01260DF11D0207A938468DF81C6039
:1019B0008DF81DB001F024FA9DF81C30002B40F08A
:1019C000A380204601F0FEFE0546002843D1704F5B
:1019D00001F0BCFB3B6898423DD301F0B7FB824667
:1019E000FFF7B4FB4FF4C8730AF5167AB0FBF3F2B5
:1019F00002FB13001AFA80F03860664F97F800B0C7
:101A0000BBFA8BF3CBF1100A5FFA8AFA5B090EA8D6
:101A10008DF82830FFF7F6FBBAF1060F28BF4FF01C
:101A2000060A0EAB03EB0B0152460DF1290000F044
:101A3000D9F90AAB0393182302930AF10102564B1A
:101A4000D2B2CDE90063049220464DA3D3E900232E
:101A500001F0FCFE3D7001F079FB504A504D1368D7
:101A6000C31AB3F57A7F2ED3106001F071FB0246E2
:101A70000B46204601F082FF204601F0A3FE10B382
:101A80002B7A484E002B0CBF02230323737101F005
:101A90005DFB0EAF4FF47A730122B0FBF3F03946D1
:101AA0003060304600F0D8FA182302933E4B019381
:101AB00080B240F25513CDE90370009342464B4685
:101AC000204601F0C3FE2B7A93B101F03FFB0026C4
:101AD00007464FF48A7A95F8D900304400F00300A5
:101AE0000AFB005393F8E82092B30136042EF2D19A
:101AF000C82002F0BDFF2B7A002B7FF43FAF13B05C
:101B0000BDEC028BBDE8F08FDAF8143083F00203ED
:101B1000CAF81430594610220EA800F06FF90DF1E2
:101B20001E0308AA0AA9384600F0F6FE95E803004D
:101B30000FAB83E803009DF834308DF844300A9BE6
:101B40000E930EA9DDE90823204602F0E7F823E70B
:101B5000D3F8E02042B12B68FA2B38BFFA23BA1A27
:101B60000533B2EB430FC0D3FFF71AFC0028BCD1FA
:101B7000BEE700BFAFF300800000000000000000DF
:101B8000401DA12026812A0BDC380020F017002000
:101B9000DC170020D8170020EC170020A01200202E
:101BA000A8120020E0170020A4120020F1C6A7C14F
:101BB000D068080F0004004808B5054800F046FF4B
:101BC000BDE80840034A0449002003F0D9BC00BF27
:101BD000F0170020603900200D15000870B5104B7B
:101BE0001B780133DBB2012B05460C4611D80D4B97
:101BF000186801684FF47A730E6AA2FB0332294613
:101C00002246B047844204D1074B00221A700120BB
:101C100070BD4FF4FA7002F02BFF0020F8E700BF10
:101C2000681100206C1100203C39002007B500230A
:101C3000024601210DF107008DF80730FFF7CEFFB6
:101C400020B19DF8070003B05DF804FB4FF0FF30B2
:101C5000F9E7000008B50A460421FFF7BFFF013885
:101C600008BD000030B4074B0A461978064B0546FC
:101C700053F821000368DC69044B2946A44630BCB4
:101C8000604700BF3C3900206C110020A086010095
:101C900070B503F0A3F8094E094C30800025206888
:101CA0003388834208D903F095F82368054401334B
:101CB000B5F5803F2360F2D370BD00BF34390020FA
:101CC0003839002003F038B900F1006000F58030A9
:101CD0000068704700F10060920000F5803003F06A
:101CE000BBB80000054B1A68054B1B889B1A834242
:101CF00002D9104403F06EB8002070473839002034
:101D000034390020024B1B68184403F069B800BF47
:101D100038390020024B1B68184403F075B800BF27
:101D2000383900200020704700F10050A0F5104025
:101D3000D0F8900570470000064991F8243033B17F
:101D40000023086A81F824300822FFF7C3BF01206E
:101D5000704700BF0C390020014B1868704700BF66
:101D6000002004E010B501380E4A0B180E48126826
:101D70000488C2F30B0294420ED142680846013A2D
:101D800098420CD212F9014F1CB92C2300F8013BE8
:101D900005E000F8014BF3E799420846F5D3401AF5
:101DA00010BD00BF002004E070110020022804BF15
:101DB000014B9861704700BF00040048022802BF31
:101DC000024B4FF400329A61704700BF0004004894
:101DD000022801BF024A536983F00203536170472E
:101DE0000004004810B50023934200D110BDCC5C24
:101DF000C4540133F8E70000FFF7FEBF0244034676
:101E0000934200D1704703F8011BF9E72DE9F8432D
:101E10001F4D144695F824200746884622B9DFF85E
:101E200070906CB9012009E02B6A03EB82038342B6
:101E3000F5D0FFF781FF0028F1D10020BDE8F8833D
:101E400095F824302BB92022FF2148462F62FFF756
:101E5000D5FF95F82400C0F10802A24228BF22460F
:101E6000D6B24146920005EB8000FFF7BBFF95F824
:101E70002430A41B1E44F6B2082E17449044E4B24A
:101E800085F82460CDD1FFF757FF0028C9D1D4E7EA
:101E90000C390020024B1A78024B1A70704700BFB1
:101EA0003C3900206811002003494FF461430B6066
:101EB000024B186802F0B8BC403900206C110020B9
:101EC00038B5094C0546182200212046FFF796FF39
:101ED000064B25601A78064B214653F82200BDE8D0
:101EE000384002F0A1BC00BF403900203C3900203E
:101EF0006C1100202DE9F3470D4604460021904661
:101F0000284640F27912FFF779FF2346202200216C
:101F1000284601F0A1FE231D02222021284601F0BF
:101F20009BFE631D03222221284601F095FEA31D7E
:101F300003222521284601F08FFE04F10803102218
:101F40002821284601F088FE04F1100308223821D8
:101F5000284601F081FE04F11103082240212846A1
:101F600001F07AFE04F1120308224821284601F00C
:101F700073FE04F1140320225021284601F06CFE68
:101F800004F1180340227021284601F065FE04F197
:101F900020030822B021284601F05EFE04F121034F
:101FA0000822B821284601F057FE04F12207C02676
:101FB0003B46314608222846083601F04DFEB6F56C
:101FC000A07F07F10107F3D194F832308DF8073084
:101FD00031460DF107030822284601F03DFE002698
:101FE00004F1330A9DF807304FEAC6099E4209F50D
:101FF000A47720D394F83231502B28BF50238DF88A
:102000000730B8F1000F08D139460DF10703072258
:10201000284601F021FE09F24F17002604F233147E
:102020009DF807309E4207EBC6010DD30731C80863
:1020300002B0BDE8F0870AEB0603082239462846BD
:1020400001F00AFE0136CDE7A3190822284601F067
:1020500003FE0136E4E7000038B50C4600210546D2
:1020600021600346C4F803102046202201F0F4FD4D
:102070002B1D20460222202101F0EEFD6B1D204683
:102080000322222101F0E8FDAB1D20460322252179
:1020900001F0E2FD204605F108031022282101F09D
:1020A000DBFD072038BD0000F7B5057F04460E466E
:1020B0002DB1838A122B02D9012003B0F0BD002379
:1020C000194607220096204601F092FC731C0093EB
:1020D000012200230721204601F08AFCD5B9B31C58
:1020E000009305222B460821204601F081FC0D2596
:1020F000B378102BE0D83746B278BB1B934210D38D
:10210000237FA08A0735ED08B3B9A8422CBF002071
:102110000120D2E7A38ADB00083BDB08B370082567
:10212000E6E7FB1C0093294600230822204601F025
:102130005FFC08350137DFE7401B18BF0120BCE713
:10214000F7B5047F05460E462CB1838ACA2B02D907
:10215000012003B0F0BD002300960822194628464E
:1021600001F046FCDCB9731C08220093114623469B
:10217000284601F03DFC10247378C82BE8D80123D1
:1021800072785F1C013B934210D32B7FA88A0734DF
:10219000E408B3B9A0422CBF00200120D9E7AB8AE4
:1021A000DB00083BDB0873700824E5E7F3190093B4
:1021B000214600230822284601F01AFC08343B4639
:1021C000DEE7001B18BF0120C3E70000F7B50E468D
:1021D00004460021154630468122FFF70FFE2346B4
:1021E00008220021304601F037FD63787F2B28BF9D
:1021F0007F238DF807309DB90DF1070307220821D1
:10220000304601F029FD0F27002502349DF80730E4
:102210009D4207EBC50105D30731C80803B0F0BDE7
:102220000827F1E763190822304601F015FD013552
:10223000ECE70000F7B50E4605460021144630468F
:10224000CE22FFF7DBFD2B4628220021304601F08D
:1022500003FD2B7AC82B28BFC8238DF807308CB913
:102260000DF1070308222821304601F0F5FC302447
:102270002F469DF807207B1B934205D3E01DC00825
:1022800003B0F0BD2824F3E707F109032146082233
:10229000304601F0E1FC08340137EAE7F7B5047F86
:1022A00005460E4634B1838AB3F5827F02D90120F8
:1022B00003B0F0BD0096012310220021284601F052
:1022C00097FBDCB9B31C0093092223461021284652
:1022D00001F08EFB19247388B3F5807FE7D8374669
:1022E0007288BB1B934210D32A7FAB8A0734E40861
:1022F000B2B99C4294BF00200120D9E7AB8ADB0031
:10230000103BDB0873801024E5E73B1D009321465A
:1023100000230822284601F06BFB08340137DFE771
:10232000E01A18BF0120C3E730B5094D0A449142B5
:1023300000D130BD11F8013B5840082340F30004A0
:10234000013B2C4013F0FF0384EA5000F6D1EEE786
:102350002083B8EDF7B5364A106851686B4603C361
:102360006A46344934480823FEF756FA044618B33F
:102370000369B3F5403F54D8418B40F28D429142FE
:1023800051D12E4A024402F110018B424DD3103B31
:10239000294900209D1AFFF7C7FF2A46064604F187
:1023A00018010020FFF7C0FFA3689E4202D1E36836
:1023B000984232D00D2500E00A25214A1068516864
:1023C0006B4603C36A461F491B480823FEF724FADD
:1023D000044618B30369B3F5403F1FD8B0F8661040
:1023E00040F28D42914219D1144A024402F15C013B
:1023F0008B4213D35C3B104900209E1AFFF794FFD9
:102400003246074604F164010020FFF78DFFA36800
:102410009F4203D1E368984200D10025284603B0CB
:10242000F0BD0B25C9E70C25C7E71025C5E700BFA0
:10243000C0550008DCFF0200000001080800FFF79B
:10244000C955000890FF020010B5037C044613B97B
:102450000068FDF7D9FF204610BD00000023BFF340
:102460005B8FC360BFF35B8FBFF35B8F8360BFF392
:102470005B8F7047BFF35B8F0068BFF35B8F704764
:1024800070B505460C30FFF7F5FF05F10806044668
:102490003046FFF7EFFFA04206D930466D68FFF7E0
:1024A000E9FF2544281A70BD3046FFF7E3FF201AE4
:1024B000F9E7000070B50546406898B105F10800DD
:1024C000FFF7D8FF05F10C0604463046FFF7D2FFB0
:1024D0008442304694BF6D680025FFF7CBFF013C76
:1024E0002C44201A70BD000038B50C460546FFF795
:1024F000C7FFA04210D305F10800FFF7BBFF6B68D0
:10250000BFF35B8F0444B4FBF3F203FB1244AC60F3
:102510000120BFF35B8F38BD0020FCE72DE9F041BF
:10252000144607460D46FFF7C5FF844228BF044600
:10253000D4B1B84658F80C6B4046FFF79BFF0644F1
:102540002E6040467E68FFF795FF331A9C4203D801
:102550006C600120BDE8F0816B60A61B3B68AB603E
:102560003044E8600220F5E72046F3E738B50C4632
:102570000546FFF79FFFA04210D305F10C00FFF7BF
:1025800079FF6B68BFF35B8F0444B4FBF3F203FB8A
:102590001244EC600120BFF35B8F38BD0020FCE7E4
:1025A0002DE9F04385B0884669460746FFF7B6FF38
:1025B0006C4606B204EBC6060025B44207D1294694
:1025C0003846FFF7D3FF284605B0BDE8F083D4F8BE
:1025D000049054F8080B08EB05014A46FFF702FC8B
:1025E0004D44EAE7F8B505460C300F46FFF742FFC9
:1025F00005F1080604463046FFF73CFFA04230468E
:1026000088BF6C68FFF736FF201A386020B130466B
:102610002C68FFF72FFF2044F8BD000073B5144667
:1026200006460D46FFF72CFF844228BF0446DCB166
:1026300001A93046FFF7D6FF019B3BB93268C5E9D7
:102640000233C5E90024012002B070BD9C4238BFAE
:102650000194019B28609C426B60F4D93268AA60A7
:10266000E41AEC600220EFE72046EDE72DE9FF4198
:102670000F466946FFF7D2FF6C4605B204EBC5056D
:102680000026AC4203D1304604B0BDE8F081D4F856
:10269000048054F8081BB8194246FFF7A3FB4644D0
:1026A000EFE7000038B50546FFF7E0FF04460146B6
:1026B0002846FFF719FF204638BD00000121884257
:1026C00038BF0846FDF77EBE08B1FDF79DBE7047D6
:1026D00003685B68184700000020704770470000DF
:1026E0000020704700F5805090F8D800C0F34000FB
:1026F0007047000000F5805090F9E000704700003E
:1027000000F58050C0F8DC1001207047F7B50C6868
:10271000BDF8207014F0005473D10D7B082D70D8D3
:10272000302585F31188056AAE6876010CD4AC6853
:10273000240108D4AC6814F0805460D184F311886B
:10274000204603B0F0BD01240E6804F1180C002EE1
:10275000B8BFF6004FEA0C1CB4BF46F0040676057D
:1027600045F80C600E680FFA84FC16F0804F18BF15
:1027700005EB0C1E05EB0C1C1EBFDEF8806146F05D
:102780000206CEF880610E7BCCF8846105EB04155F
:102790008E68C5F88C614E68C5F88861DCF8805198
:1027A00045F00105CCF8805141F2780500EB441C5E
:1027B000660105EB4414AC440444CCE900230D4607
:1027C000083401F10C0C55F804EB44F804EB6545B2
:1027D000F9D12D882580841904F5805407F003056C
:1027E00094F8946026F00B06354384F89450002446
:1027F00084F31188009700F0FDFC0120A1E702247A
:10280000A2E74FF0FF309CE738B500F580540D4645
:10281000E06EFFF74FFE1F2809D9E06E20222946FF
:10282000FFF7BEFEA0F120035842584138BD0020FA
:10283000FCE7000008B5302383F3118800F58050D1
:10284000C06EFFF70BFE002383F3118808BD000064
:1028500000220260828142608260704710B50022CF
:102860000023C0E900230023044603810C30FFF756
:10287000EFFF204610BD0000F0B5054600F5805082
:102880000C4690F8D83013F0040FC3F3800108BF52
:10289000114661F3820380F8D83005EB441303F549
:1028A0008453103389B01B79D8074FEA44162FD5CB
:1028B00082B319072ED46846FFF7D0FF05EB441307
:1028C00003F5845303AA03F10807186859681446EE
:1028D00003C40833BB422246F7D1186820609B88A6
:1028E000A380DDE90E23CDE900230123ADF80830F4
:1028F0002B6869469B6B28469847354405F58455F7
:1029000010352B791A075CBF43F008032B7101E0E7
:10291000002AF2D109B0F0BD2DE9F0479A4688B0FF
:10292000074688469146302383F3118807F5805483
:102930006846FFF793FFE06EFFF7A2FD1F282AD934
:10294000E06E20226946FFF7ADFE202823D103ADBB
:10295000444605AB2E4603CE9E422060616035465C
:1029600004F10804F6D130682060B388A380DDE963
:102970000023C9E90023BDF80830AAF8003000237D
:1029800083F3118853464A464146384608B0BDE8AD
:10299000F04700F0E9BB002080F3118808B0BDE8E3
:1029A000F08700002DE9F84F182204460F46043046
:1029B0000021FFF723FA2046214B40F8243BFFF784
:1029C00047FF04F13800FFF749FF04F1580804F508
:1029D00082554646183530462036FFF73FFFAE4257
:1029E000F9D104F580554FF48053C5F858804FF065
:1029F0000008C5E917380123EE66C5F8648085F83C
:102A0000683085F8703004F5845604F587594FF026
:102A1000000A4FF0000B46E902AB3046FFF718FF03
:102A2000203646F8108C4E45F5D185F8E07017B188
:102A3000044800F085FB044B23622046BDE8F88F74
:102A4000FC550008D25500080064004010B5044B46
:102A5000197804464A1C1A70FFF7A4FF204610BDDF
:102A6000583900202DE9F04711B90020BDE8F08762
:102A7000274B284EB6FBF1F4994294BF11230A2349
:102A8000013BDBB2581CB4FBF0FC00FB1C405FFABE
:102A900083FEC0BB0CF1FF37B7F5806FE5D2C3EB07
:102AA000C303D81C4FEAE009C0F3C700AEEB00082F
:102AB00009F1010A4FF47A755FFA88F409FB0555AC
:102AC0005AFA88F8B5FBF8F5B5F5617FC1BF03F197
:102AD000FF33C3F3C700AEEB0003DCB2431C54FA70
:102AE00083F30CFB03F3B6FBF3F68E42BDD1013C3E
:102AF000E4B2072CB9D801380023D0701780937046
:102B000014710120B2E7BEF1020FAED0013BB9E76C
:102B10003F420F0000B4C40470B505460E464FF4A2
:102B20007A742B6A5B6803F00103B34207D04FF459
:102B30007A7001F09DFF013CF3D1204670BD012069
:102B4000FCE7000030B5026A936913F0700F17D0EC
:102B50000023936141F2900400EB43122244117967
:102B60004D070AD5890708D5064D016A55F8235047
:102B70008D60117941F0040111710133032BEBD108
:102B800030BD00BF3856000873B51D46036A1646AF
:102B90009A68D207044609D59A6801219960C2F360
:102BA0004002CDE900650021FFF766FE236A9A68BE
:102BB000D1050BD59A684FF480719960C2F3402219
:102BC000CDE9006501212046FFF756FE236A9A6889
:102BD000D2030BD59A684FF480319960C2F340421A
:102BE000CDE9006502212046FFF746FE04F580533B
:102BF000D3F8DC0010B103681B699847204602B087
:102C0000BDE87040FFF79EBFF8B50446066A00298C
:102C100077D106F10C073868800775D006EB0115EF
:102C20003868D5F8B00110F0040FD5F8B0011ABF1C
:102C3000C00840F00040400D6062D5F8B0C11CF003
:102C4000020F1CBF40F080406062D5F8B40106EB73
:102C5000011100F00F0084F83000D1F8B80184F8B9
:102C60002800D1F8B801000A84F82900D1F8B80189
:102C7000000C84F82A00D1F8B801000E84F82B006B
:102C8000D1F8BC0184F82C00D1F8BC01000A84F80A
:102C90002D00D1F8BC01000C84F82E00D1F8BC1135
:102CA000090E84F82F103821396004F1440004F132
:102CB000240104F1300551F8046B40F8046BA9427B
:102CC000F9D109880180C4E90E2321460023A4F824
:102CD000403051F8383B20469B6B984704F58053B1
:102CE00093F8D820D3F8DC0042F0040283F8D8200F
:102CF00010B103681B6998472046BDE8F840FFF70C
:102D000021BF06F1100786E7F8BD000010B50446A4
:102D100000F01EFA02460B4652EA030102D0013AC5
:102D200063F100030449086820B12146BDE8104062
:102D3000FFF76ABF10BD00BF5C390020F0B530213D
:102D400081F3118800F583511831002441F2900C71
:102D500000EB441565442E7977070FD4F6060DD5A0
:102D6000D1E9007697429E4108D2094F066A57F88A
:102D70002470B7602E7946F004062E710134032CBE
:102D800001F12001E4D1002383F31188F0BD00BFDD
:102D90003856000808B5302383F31188FFF7D2FEB8
:102DA000002383F3118808BD036A9B6813F0E05F7A
:102DB00014BF01200020704708B5302383F3118829
:102DC00000F58050C06EFFF75BFB002383F3118892
:102DD00040090CBF0120184608BD0000F8B51E468A
:102DE000002313700F4605461446FFF7E5FF80F0F9
:102DF000010038701EB12846FFF7D6FF2070F8BDDD
:102E0000F8B50C4615461E46074600F0A1F90B46DC
:102E10002178024609B9287850B13846FFF78EFF6D
:102E2000FFF7B8FF33462A462146FFF7D7FF0120B8
:102E3000F8BD000070B5302686F31188174B9A6DE7
:102E400042F000729A659A6B42F000729A639A6B34
:102E500022F000729A63002383F3118800F58054F6
:102E600094F8D83013F0010516D1A9B186F3118872
:102E70000321132001F020FB0321142001F01CFB8F
:102E80000321152001F018FB94F8D83043F001031A
:102E900084F8D83085F3118870BD00BF001002405F
:102EA0002DE9F04300F5805589B095F8E030012B0D
:102EB00004460F4676D8DFF8EC8158F823200AB98B
:102EC00048F82300D8F80090E761B9F1000F0BD162
:102ED00041F2E800FFF7F2FB0646002860D04946C1
:102EE000FFF760FDC8F8006095F8E030012B5DD079
:102EF00001212046FFF79EFF302383F31188226AC9
:102F0000136823F002031360226A136843F001037D
:102F10001360236A00265E6186F311880121204632
:102F2000FFF7FAFD00287DD0E86EFFF797FA04F569
:102F3000835808F11808202200216846FEF75EFF3A
:102F400002A8FFF785FC6A4608EB06030DF1180E90
:102F50009446BCE80300F44518605960624603F1EA
:102F60000803F5D1DCF80000186020369CF8042036
:102F70001A71602EDFD195F8D83023F0040385F85C
:102F8000D83000266A463946204600968DF80460FF
:102F9000FFF768FD236AF0B94FF400421A6001E0C0
:102FA000C8F80000002009B0BDE8F083D8F80000A0
:102FB00003689B6A98470146002899D1D8F8000019
:102FC000FFF738FFD8F80000036839465B68984778
:102FD00000288DD1E6E765221A609DF803109DF860
:102FE0000230226A1B06090401F4702103F04073C9
:102FF0000B43BDF80010C1F309010B439DF8041009
:10300000090501F4E0010B43D361236A13225A61DD
:10301000226A136823F00103136031462046FFF74C
:103020007BFD08B9236AB7E795F8E02092BB216AD7
:10303000D1F8003243F00103C1F80032216AD1F81F
:10304000003223F47C5323F00E03C1F80032216ACE
:10305000D1F8003243F46063C1F80032236AC3F848
:103060001422236AC3F80422236A41F6FF71C3F8CD
:103070000C12236AC3F84022236AC3F84422236A4D
:103080000122C3F81C22226AD2F8003223F0010385
:10309000C2F8003295F8D83043F0020385F8D830F2
:1030A00081E700BF5C39002008B500F051F8024606
:1030B0000B4652EA030102D0013A63F100030449CE
:1030C000086808B1FFF760FDBDE8084001F0A6B848
:1030D0005C39002008B50020FFF718FEBDE8084065
:1030E00001F09CB808B50120FFF710FEBDE80840CC
:1030F00001F094B800B59BB0EFF3098168226846EF
:10310000FEF770FEEFF30583014B9B6BFEE700BFFC
:1031100000ED00E008B5FFF7EDFF000000B59BB043
:10312000EFF3098168226846FEF75CFEEFF3058342
:10313000014B5B6BFEE700BF00ED00E0FEE7000027
:103140000FB408B5029801F043FCFEE701F038BF68
:1031500001F01ABF0139C9B202299EBF00EBC100BC
:103160000023C0E9013370472DE9F8431E461B8850
:103170005B070546884605D400F10C0400F12409DC
:10318000A14502D10120BDE8F88354F8083C13B9E9
:1031900054F8043C6BB12B6828465B6B9847338826
:1031A00054F8047CC1B243F0040354F8080C4246BE
:1031B000B8470834E4E7000073B56C4684E80600BD
:1031C000014600224E68551C66B98E6856B900EB60
:1031D000C200021D94E8030082E803001D70012074
:1031E00002B070BD032D2A4601F10801EAD100208A
:1031F000F6E700002DE9F04F89B00446BDF848809D
:103200008B4600F10C0500F12409002708F0040AA0
:10321000A94503D1012009B0BDE8F08F55F8083C5D
:1032200013B955F8043C63B1BAF1000F0BD1236810
:1032300020465B6B98474346C1B25A4655E90206A1
:10324000B0470835E4E70FBB00220023CDE9002397
:10325000ADF808705B4603AA0BF1080C18685968B2
:10326000174603C7083363453A46F7D118683860F4
:103270009B88BB80FFF76CFF0423ADF80830236800
:10328000CDE900019B6B6946204698470127D8E7A6
:103290000E2809D8DFE800F01515151515151515B8
:1032A000150A0C0E10121400402070470C207047B5
:1032B0001020704714207047182070472020704756
:1032C000302070472DE9F043456A35B94162BDE8C9
:1032D000F083CEF800100B60F9E74E6826F0604CE2
:1032E000C6F38A47C6F3807817EA260738BF6746D1
:1032F000AE462B465C6894EA060F24F060420CD57B
:10330000002C1EDA920CBA4201D0BA420FD99D426B
:10331000DFD10D60DAE71346ECE7944505D104F000
:103320008049C4F38074444507D19445EFD31A68AB
:103330009E46002AEFD11960C9E7B9F1000FF6D017
:10334000E5E7BA42F3D0E0E72DE9F047089E01F047
:1033500007054FEAD6082A4406F0070600EBD1011C
:103360004FF47F49954201D1BDE8F08705F0070C85
:1033700006F0070AD445674638BF5746C7F1080725
:10338000501BEC08874228BF07460C5D08EBD600AF
:1033900004FA0CF413F800E029FA07FC24FA0AF402
:1033A0005FFA8CFC8EEA04044CFA0AFC04EA0C0472
:1033B0008EEA040E03F800E03D443E44D2E70000EC
:1033C00080EA0120082341F2210201B240000029D5
:1033D00080B203F1FF33B8BF504013F0FF03F4D1C4
:1033E0007047000038B50C468D18A54200D138BD95
:1033F00014F8011BFFF7E4FFF7E7000003464068FD
:1034000048B102685A605A899989013292B2914250
:103410005A8138BF9A81704770B588B0202204461F
:103420000D4668460021FEF7E9FC20460495FFF7AB
:10343000E5FF024658B16B46054608AE1C4603CC74
:10344000B44228606960234605F10805F6D11046AC
:1034500008B070BD2DE9F843078C072F04461ED92C
:10346000D0E9029800254FF6FF73C5F12006A5F1BB
:10347000200029FA05F108FA06F628FA00F031438F
:103480000143C9B21846FFF79BFF0835402D03469C
:10349000EBD1E1693A46BDE8F843FFF7A3BF4FF629
:1034A000FF70BDE8F883000010B54B6823B9CA8AE5
:1034B00063F30902CA8210BD04691A681C600361C3
:1034C000C38A013BC3824A60EFE700002DE9F84F51
:1034D0001C46CB8A8046C3F3090005280F46914657
:1034E00003462ED000221A319DB2042D96B211D877
:1034F000B44203F1010308D80444FB8AC4F309046D
:1035000064F30903FB82012019E019F80250CD543D
:103510000132E9E7B442EFD9A0F1050A1C237D6826
:10352000BAFBF3F203FB12AA1FFA8AF295BB4046DC
:10353000FFF764FF054630B978606FF00200BDE820
:10354000F88F0026E8E70022026078604FF0000A5A
:10355000B44242D9D31C2B44901B25E0013189B2DF
:103560001D462B68002BF9D1631F03441C20B3FBBD
:10357000F0F301339BB29942E8D2BAF1000FE5D1E2
:103580004046FFF73BFF38B1C0F800A05246286024
:103590000546DBE70121E4E7C5F800A0CDE719F80F
:1035A000061003F8011F013610FA86F189B21B29B3
:1035B0001FFA86FB03D85C45F1D85E46C8E75C4538
:1035C000FBD94046FFF71AFF28B1C0F800A000223F
:1035D00028600546F1E72860AFE7FB8A1C448CE7CA
:1035E0002DE9F74F1C465B69009207468846002B81
:1035F00000F0B580238C2BB1E269002A00F0AF8087
:10360000072B4AD807F10C00FFF7F8FE054620B952
:103610006FF0020003B0BDE8F08F14220021FEF726
:10362000EDFB228CE16905F10800FEF7DBFB208C45
:10363000013080B208280DD90C2824D9102824D9AB
:10364000142824D9182824D9202824D9312834BF73
:103650000E200F20FFF71CFE013880B220840130BD
:1036600028746369228C1B782A4403F01F0363F0DB
:103670003F03137248F0004338466B602946FFF75A
:1036800021FE0120C6E70920E4E70A20E2E70B203B
:10369000E0E70C20DEE70D20DCE702339BB20722D7
:1036A000C18A0633B3FBF2F3828A521A9BB292B2FA
:1036B0009342ADD8002500F10C034FF08009AA46D3
:1036C0002E460193238CB34201D128B2A2E7019880
:1036D000FFF794FE834600289AD014220021FEF7BB
:1036E0008DFB56B9009BABF8083002220BF1080C99
:1036F000218CB14203D890B20BE00022F6E7E169D9
:10370000895D0CF80210013290B201360728B6B27A
:10371000EED1228C013080B2FFF7BAFDB24208BF71
:103720004FF0400962691278013802F01F021BFA5B
:1037300080F142EA4A1249EA02020A72013048F074
:1037400000428BF81000CBF8042059463846FFF7AA
:10375000B9FD8AF0010A01354FF00009B2E76FF0B8
:10376000010057E7F8B515460E4630220021044601
:103770001F46FEF743FBB5F5001F069B636034BF91
:103780006A094FF6FF72079BA76095B2A362E661D4
:1037900004F1100006EB4212964206D100230360AA
:1037A000A582E3822383E360F8BD066030462036BD
:1037B000F2E7000003781BB94BB2002BC8BF0170C1
:1037C0007047000000787047F8B50C46C969074695
:1037D00009B9238CB3BB257E1F2D33D83B7823BB7F
:1037E000228C072A2BD8268A032E2BD84FF6FF705F
:1037F000FFF7F8FD20F001003602400446EA0566B6
:10380000400C46EA40254FF6FF72234629463846CB
:10381000FFF7E6FE002807DD626913780133DBB2AB
:103820001F2B88BF00231370F8BD228A2D0645EA9E
:10383000022520461D43FFF70DFE0246E5E76FF027
:103840000300F1E76FF00100EEE7000070B58AB009
:10385000044616460021282268461D46FEF7CEFA89
:10386000BDF83830ADF810300F9B05939DF840300F
:103870008DF81830119B07936946BDF84830ADF8B4
:1038800020302046CDE90265FFF79EFF0AB070BDEB
:103890002DE9F041D36905460C4616460BB9138C49
:1038A0005BBB377E1F2F28D895F80080B8F1000F3A
:1038B00026D03046FFF7CEFD3378210241EAC331EE
:1038C00041EA0801338A41EA076141EA03410246BD
:1038D000334641F080012846FFF782FE00280ADDCA
:1038E0003378012B07D1726913780133DBB21F2BB8
:1038F00088BF00231370BDE8F0816FF00100FAE784
:103900006FF00300F7E70000F0B58BB004460D46FA
:1039100017460021282268461E46FEF76FFA9DF8DA
:103920004C305A1E534253418DF800309DF84030C0
:10393000ADF81030119B05939DF848308DF8183084
:10394000149B07936A46BDF85430ADF820302946E1
:103950002046CDE90276FFF79BFF0BB0F0BD0000DB
:10396000406A00B104307047436A1A6842620269D3
:103970001A600361C38A013BC38270472DE9F84393
:10398000D0F82090194F14461E4649464FF00008C3
:1039900009B9BDE8F883D1E90252651B66EB020262
:1039A000AF4278EB02021ED2036A8B420DD1FFF7C1
:1039B0007BFD036A1B68036203690B60C38A0161B4
:1039C000016A013BC3828946E2E7FFF76DFD0B68A0
:1039D000C9F8003003690B60C38A0161013BC382EF
:1039E000D9F80010D4E789460968D1E780841E0021
:1039F0002DE9F04F8BB00D46DDF85080049314464E
:103A00008246002800F01881B8F1000F00F0148100
:103A1000531E3F2B00F21081012A03D1049B002B7F
:103A200040F00A81BAF814B00023B5EBCB0FCDE912
:103A300008334FEACB0703D300200BB0BDE8F08F6B
:103A40002B199F42DAF80C3003933ABF7F1BFFB269
:103A500027461BB9DAF81030002B75D0272D4AD82D
:103A6000C5F12806B7424FF000032CBFF6B23E4620
:103A700000932946DAF8080008AB3246FFF764FCE9
:103A8000A7EB060935445FFA89F90BF1005BABF14E
:103A9000050B4FEACB0B2821039B13B1B9F1000FA3
:103AA0002CD1DAF8100040B1B9F1000F05D0009622
:103AB00008AB4A46691AFFF747FC38B2002FBBD063
:103AC00067070AD00AAB03EBD401624211F8083C45
:103AD00002F00702134101F8083C082C3BD9102CD6
:103AE00040F2B580202C40F2AD80049B002B00F00A
:103AF0009780082332E0B9460026C6E75B46E02BF4
:103B000028BFE02306930B44AB42059314D95A1BFC
:103B100003980096914534BF4A46D2B2691A08AB61
:103B200004300792FFF710FC079A16441544A9EBDE
:103B30000202F6B25FFA82F9069B0599ABEB030B22
:103B4000039B1B680393A7E70093DAF8080008AB10
:103B50003A462946AFE7049B93B10123B4EBC30F68
:103B600063D0082C11D89DF82030621E23FA02F28F
:103B7000D60705D54FF0FF32A24013438DF8203011
:103B80009DF8203088F8003057E7102C11D8BDF888
:103B90002030621E23FA02F2D50705D54FF0FF321E
:103BA000A2401343ADF82030BDF82030A8F8003013
:103BB00043E7202C0ED8089A631E22FA03F3D90794
:103BC00004D54FF0FF33A34013430893089BC8F874
:103BD000003032E7402C32D0DDE90851631EC4F1D9
:103BE0002106A4F1210225FA03F301FA06F6334374
:103BF00021FA02F21343DB0712D50123A4F12002BC
:103C0000C4F1200603FA02F223FA06F6A3405B424F
:103C100042EA060262EB42022B430A43CDE9083234
:103C2000DDE90823C8E9002307E7082CA8D0102CF9
:103C3000BAD0202CF4D1C9E76FF00100FDE66FF097
:103C40000800FAE6049B002BC0D0042386E7049BFF
:103C5000002BA9D0022381E730B5012A144638BFD2
:103C60000122402A85B028BF40220025012CCDE941
:103C700002550ED81B788DF8083004AB03EBD20543
:103C8000544215F8083C04F00704A34005F8083C2A
:103C900006E0082C0CD81B788DF808305307ECD1BF
:103CA00000910346002102A8FFF74EFB05B030BD8E
:103CB000102C03D81B88ADF80830EFE7202C8DBFFF
:103CC000D3E900451B680293CDE90245E6E7000011
:103CD00010B5CB681BB98B600B618B8210BD04697A
:103CE0001A681C600361C38A013BC382CA60F0E7A3
:103CF00003064CBFC0F3C0300220704708B502462F
:103D0000FFF7F6FF022806D15306C2F30F2001D1B8
:103D100000F0030008BDC2F30740FBE72DE9F04FB8
:103D2000D1F8008097B004464046CDE90623FFF75E
:103D3000DFFF022814BFC8F306260026B8F1000FE3
:103D40000D46039080F2F88118F0C04A40F0F481EB
:103D5000097B002900F0F081039B022B03D023781C
:103D6000B34240F0EC8108F07F0340460493FFF734
:103D7000C5FF049B059029444FEA8349039B91F8B2
:103D800003B049EA034949EA4669002200235FEA91
:103D9000DB16CDE90C2349EA000978D0049B009397
:103DA00002466768039B0CA92046B847002800F02C
:103DB000C981276A002F58D1494604F10C00FFF74A
:103DC0002BFB0746002800F0EF8027626B7B0A93ED
:103DD000BB7E0B93FB7D0BF01F09C3F38403A3EBA6
:103DE00009001FFA80FC0028B8BF0CF1200C0890D5
:103DF000A9EB0303B8BF0FFA8CF0D7E902121FFA40
:103E000083FCB8BF0890002BB8BF0CF1200C0993BD
:103E1000BCBF0FFA8CF3099351EA020ED7F804C025
:103E200000F0A981069B591A079B63EB0202B14B74
:103E30004FF0000E8B427EEB0203C0F09C81DDE967
:103E40000A30834240F08A81002E36D0089B012B35
:103E500000F39181BCF1000F40F08D81A6488842AB
:103E60007CEB0202C0F0838130E03B699945ADD024
:103E70003F68002FF9D1494604F10C00FFF7CCFA56
:103E80000746002800F09080236A3B609DE7276A80
:103E900077B9049B00936568039B059A0CA920469B
:103EA000A847C0F57F40F43000B217B0BDE8F08FEE
:103EB0003B6999458AD03F68EAE78F4B8B4276EBA6
:103EC000020203D26A7BBB7E9A4239D1C8F30468EE
:103ED000002E37D01BF0400F34D0069BBB60079BF1
:103EE000FB601422002111A8FDF788FF069B0E93AA
:103EF000079B0F932B1D10932B7B8DF85190013B4B
:103F0000DBB2ADF84C30059BADF84E30039B8DF81D
:103F10005030049B8DF8533094F82C308DF852803B
:103F200083F001038DF854300EA9A368204698470A
:103F3000FB7DC3F38403013303F01F039B02FB8269
:103F40000020B2E7FB7DCBF34012B2EBD31F40F071
:103F5000FC80C3F384034B4540F0FA802B7B002E9A
:103F600051D0032B40F2F780069BBB60079BFB60A0
:103F7000FB8A6FF30903FB822B7BAE1D033BDBB295
:103F80003246394604F10C00FFF7A0FA00280EDA99
:103F900039462046FFF788FAFB7DC3F384030133DB
:103FA00003F01F039B02FB826FF002007DE7DDE957
:103FB0000C84AB883B834FF6FF73CAF12000AAF153
:103FC000200228FA0AF104FA00F0014324FA02F26E
:103FD00011431846C9B2FFF7F3F90AF1080ABAF11A
:103FE000400F0346E9D1B8822A7B033AD2B2314668
:103FF000FFF7F8F9FB7DB882DA43C2F3C01262F32F
:10400000C713FB759CE7013B5FEA9B1BDBB20ED13C
:104010002E1D3246394604F10C00FFF757FA0028EE
:10402000B6DB2A7BB88A013AD2B23146E0E7FA8A97
:10403000C2F30902042A61D86BB1E91C07F11B0025
:1040400011F801CF00F802C001320136052AF6B29C
:1040500001D09E42F4D3069A0E92079A0F929E4286
:1040600007F11B02109238BF04367A68119234BFF0
:1040700055FA86F600261296FA8A8DF85190C2F308
:1040800009021344ADF84C30059BADF84E30039B4C
:104090008DF85030049B8DF8533094F82C308DF807
:1040A000528083F001038DF8543000237B602A7B1B
:1040B000B88A013A291DFFF795F93B8BB8828342F4
:1040C00003D1A3680EA92046984720460EA9FFF702
:1040D000FFFDFB7DBA8AC3F38403013303F01F03A2
:1040E0009B02FB823B8B9A4214BF6FF010000020B2
:1040F000DBE600BF80841E0040420F007868002885
:10410000A9D0052101E01C3130460668002EFAD105
:10411000521AD11C05F1030C014402EB0A001B28C2
:104120005FFA8AF697D89E4295D21CF8010F01F8E3
:10413000010F0AF1010AF0E76FF00900B5E66FF030
:104140000A00B2E66FF00B00AFE66FF00D00ACE6D0
:104150006FF00E00A9E66FF00F00A6E61448884243
:104160007EEB0202BFF4ECAE002E3FF4ABAE099B37
:104170000F2B3FF7A7AEFA7D4FEA8B0302F0030245
:1041800003F07C031343FB7539462046FFF78CF997
:104190006B7BBB76002E7FF495AEFB7DC3F3840270
:1041A000013262F38603FB756FF00C007DE600BF01
:1041B00040420F00EFF3098305494A6B22F00102E8
:1041C0004A63683383F30988002383F311887047B7
:1041D00000EF00E0302080F3118862B60C4B0D4AEE
:1041E000D96821F4E0610904090C0A43DA60D3F8C4
:1041F000FC20094942F08072C3F8FC200A6842F0B2
:1042000001020A602022DA7783F82200704700BF9B
:1042100000ED00E00003FA05001000E010B53023C7
:1042200083F311880E4B5B6813F4006314D0F1EE36
:10423000103AEFF30984683C4FF08073E361094B57
:10424000DB6B236684F3098800F086FB10B1064B14
:10425000A36110BD054BFBE783F31188F9E700BFAD
:1042600000ED00E000EF00E0FF020008020300089C
:10427000026843680A43026003B1184770470000B0
:10428000024A136843F0C0031360704700380140CE
:1042900013B50E4C204600F0BBFA04F114000C4993
:1042A000009400234FF4807200F078F9094B0A491A
:1042B00000944FF4807204F1380000F0F1F9074ADD
:1042C000074BC4E9172302B010BD00BF643B0020B8
:1042D000643A00208142000864390020003801401F
:1042E00000B4C404254B30B5002914BF0C461C464D
:1042F000037C012B0FD1224B98420CD1214B1A6E1B
:1043000042F480421A66D3F8802042F48042C3F817
:104310008020D3F880302268036EC16D846603EB81
:104320005203B3FBF2F36268150442BF23F00705A2
:1043300003F0070343EA4503CB60A36843F040035F
:104340004B60E36843F001038B6042F4967343F0E3
:1043500001030B604FF0FF330B6251050AD512F0D9
:10436000102209D0B2F1805F14BFFF233F2380F8F1
:10437000643030BDFF23FAE77F23F8E74456000896
:10438000643B0020001002402DE9F047C66D3768FD
:10439000F56935622A07044618D045F30001C5F3D4
:1043A000C00301F0200141EA0321AB0748BF41F0FF
:1043B0004001680748BF41F08001302383F3118832
:1043C000201DFFF755FF002383F31188EA050AD566
:1043D000302383F311884FF48061201DFFF748FFDD
:1043E000002383F311884FF030084FF0000A0BE0F0
:1043F00088F31188B38C94F864102046194000F0BB
:1044000021FA8AF31188F56915F02009F0D13B06ED
:1044100016D54FF0300A04F13808280610D58AF373
:104420001188404600F070F9002829DA0821201D83
:10443000FFF71EFF27F080033360002383F311880A
:10444000790614D56A0612D5302383F31188D4E98E
:1044500013239A4208D1236C33B11021201D27F079
:104460004007FFF705FF3760002383F31188EB0651
:104470000CD5A26E13694BB1BDE8F04750691847DF
:1044800080B2308589F31188F569C6E7BDE8F08709
:104490004FF0E023002258684FF0FF31930003F102
:1044A000604303F5614301329042C3F88010C3F8C2
:1044B0008011F3D27047000000F1604303F56143BF
:1044C0000901C9B283F80013012200F01F039A40CA
:1044D00043099B0003F1604303F56143C3F8802166
:1044E0001A607047F8B5154682680669AA420B46FD
:1044F000816938BF8568761AB54204460BD22A46D0
:104500001846FDF76FFCA2692A44A368A2615B1BF1
:10451000A3602846F8BD0CD918463246FDF762FC68
:10452000AF1B3A46E1683044FDF75CFCE368DA19FA
:10453000EBE72A461846FDF755FCE268E5E7000080
:10454000836893422DE9F0411546044638BF8568DB
:10455000D0E904703F1ABD420E460BD22A46FDF741
:1045600041FC62692A44A36862615B1BA360284620
:10457000BDE8F0810DD93A46A5EB0708FDF732FCFE
:104580004246E068F119FDF72DFCE36803EB0802F1
:10459000E9E72A46FDF726FCE268E4E710B5C0E942
:1045A00005110024C160C3611144029B8460C0E90D
:1045B00000000161036210BD08B5D0E905329342E5
:1045C00001D1826882B98268013282605A1C4261DC
:1045D0001970D0E904329A4224BFC36843610021B4
:1045E00000F062FA002008BD4FF0FF30FBE700004A
:1045F00070B5302304460D4683F31188A668A6B132
:10460000A368A269013BA360531CA36115782269CA
:10461000934224BFE368A361E3690BB12046984746
:10462000002383F31188284607E02946204600F03E
:104630002BFA0028E2DA86F3118870BD2DE9F74FD6
:1046400005460F4614469946D0F81CA04FF0300896
:1046500088F311884FF0000B164666B13246394692
:104660002846FFF73FFF034660B94946284600F059
:104670000BFA0028F2D0002383F31188A01B03B0AB
:10468000BDE8F08FBAF1000F03D001902846D04763
:10469000019B8BF31188F61A1F4488F31188DCE71D
:1046A000C0E90511C160C3611144009B8260C0E98B
:1046B0000000016103627047F8B504460D461646D6
:1046C000302383F31188A768A7B1A368013BA360D7
:1046D00063695A1C62611D70D4E904329A4224BF96
:1046E000E3686361E3690BB120469847002080F3DB
:1046F000118807E03146204600F0C6F90028E2DACA
:1047000087F31188F8BD0000D0E905239A4210B55F
:1047100001D182687AB98268013282605A1C826152
:104720001C7803699A4224BFC3688361002100F0AA
:10473000BBF9204610BD4FF0FF30FBE72DE9F74FE6
:1047400005460F4614469946D0F81CA04FF0300895
:1047500088F311884FF0000B164666B13246394691
:104760002846FFF7EDFE034660B94946284600F0AB
:104770008BF90028F2D0002383F31188A01B03B02B
:10478000BDE8F08FBAF1000F03D001902846D04762
:10479000019B8BF31188F61A1F4488F31188DCE71C
:1047A000026843680A43026003B11847704700007B
:1047B0001430FFF743BF00004FF0FF331430FFF712
:1047C0003DBF00003830FFF7B9BF00004FF0FF33A6
:1047D0003830FFF7B3BF00001430FFF709BF000007
:1047E0004FF0FF311430FFF703BF00003830FFF700
:1047F00063BF00004FF0FF323830FFF75DBF0000AD
:10480000012914BF6FF0130000207047FFF740BD6F
:10481000044B03600023C0E90233436001230374A7
:10482000704700BF5C56000810B53023044683F380
:104830001188FFF757FD02232374002080F31188AD
:1048400010BD000038B5C36904460D461BB90421EC
:104850000844FFF7A5FF294604F11400FFF7ACFE5A
:10486000002806DA201D4FF40061BDE83840FFF74C
:1048700097BF38BD00230375826803691B68996878
:104880009142FBD25A6803604260106058607047E2
:1048900000230375826803691B6899689142FBD8FD
:1048A0005A680360426010605860704708B5084657
:1048B000302383F311880B7D032B05D0042B0DD0FF
:1048C0002BB983F3118808BD8B6900221A604FF061
:1048D000FF338361FFF7CEFF0023F2E7D1E9003217
:1048E00013605A60F3E70000FFF7C4BF38B50A4B06
:1048F000DD681C68287522681A605360DC60A36854
:1049000001229342227501D100F01CFC2946204669
:10491000BDE83840FBF7DEBCE03D002030B50C4B75
:10492000DD684B1C87B004460FD02B46094A684609
:1049300000F04CF92046FFF7D9FF009B13B1684601
:1049400000F04EF9A86907B030BDFFF7CFFFF9E7D7
:10495000E03D0020AD480008044B1A68DB68906811
:104960009B68984294BF002001207047E03D0020E2
:1049700038B50B4B1C68DD6822681A605360012251
:104980002275DC60AB68934201D100F0DDFB284664
:10499000FFF77EFF01462046BDE83840FBF79ABC92
:1049A000E03D002038B5074C0749084801230025A1
:1049B0002370656000F006FC0223237085F31188E4
:1049C00038BD00BF383E002084560008E03D00207E
:1049D00008B572B6044B186500F0C2FA00F070FB1F
:1049E000024B03221A70FEE7E03D0020383E002013
:1049F00000F02CB98B60022308618B820846704757
:104A00008368A3F1840243F8142C026943F8442C10
:104A1000426943F8402C094A43F8242CC26843F801
:104A2000182C022203F80C2C002203F80B2C044A49
:104A300043F8102CA3F12000704700BFED020008DE
:104A4000E03D002008B5FFF7DBFFBDE80840FFF7B9
:104A50004BBF0000024BDB6898610F20FFF746BF99
:104A6000E03D0020302383F31188FFF7F3BF0000FF
:104A700008B50146302383F311880820FFF74EFF65
:104A8000002383F3118808BD064BDB6839B1426807
:104A900018605A60136043600420FFF73FBF4FF077
:104AA000FF307047E03D002003460068834205D098
:104AB00002681A6053608161FFF716BF70470000FB
:104AC00010B503689C68A2420CD85C688A600B60D1
:104AD0004C60216059609968891A99604FF0FF33E2
:104AE000836010BD1B68121BECE700000A2938BF69
:104AF0000A2170B504460D460A26601900F05CFBD9
:104B000000F048FB041BA54203D8751C2E46044642
:104B1000F3E70A2E04D9BDE87040012000F092BBF3
:104B200070BD0000F8B5144B1446D961826003F1E2
:104B3000100242600A2C1A69026038BF0A245060D1
:104B4000186108190D4600F029FB0A2700F022FB26
:104B5000431BA342064606D37C1C281900F02CFBFD
:104B600027463546F2E70A2F04D9BDE8F840012070
:104B700000F068BBF8BD00BFE03D002070B50D46F9
:104B8000064600F007FB0F490B4653F8102F9A42D8
:104B900006D12A4601463046BDE87040FFF7C2BF45
:104BA000CB69C41A2C19936828BF2C46A34202D99A
:104BB0002946FFF79BFF224631460348BDE8704077
:104BC000FFF77EBFE03D0020F03D002010B4C0E9BB
:104BD000032300235DF8044B4361FFF7CFBF0000C0
:104BE00010B5194C236998420DD0D0E90032816884
:104BF00013605A609A680A449A60002303604FF079
:104C0000FF33A36110BD2346026843F8102F5360A1
:104C10000022026022699A4203D1BDE8104000F0F0
:104C2000C5BA936881680B44936000F0B3FA2269B7
:104C3000E1699268441AA242E4D91144BDE81040E7
:104C4000091AFFF753BF00BFE03D00202DE9F047F0
:104C5000DFF8B88008F110072B4ED8F8105000F09C
:104C600099FAD8F81C40AA68011B8A423DD814441E
:104C7000D5E90032C8F81C4013605A6000232B604D
:104C8000D8F81020B242994601D100F08FFA89F38A
:104C90001188D5E9033128469847302383F31188DA
:104CA0006B69002BD9D000F075FA6A69A0EB040992
:104CB0004A4582460DD2022000F0C4FA0022D8F8FC
:104CC0001030B34208D151462846BDE8F047FFF7FF
:104CD00029BF2244121AF2E712EB090938BF4A46EB
:104CE00029463846FFF7ECFEB6E7D8F81010B14277
:104CF00008D01444211AC8F81C00A960BDE8F04788
:104D0000FFF7F4BEBDE8F087F03D0020E03D002055
:104D100038B500F03FFA054AD2E90845031B1819D7
:104D200045F10001C2E9080138BD00BFE03D0020A7
:104D300000207047FEE70000704700004FF0FF3092
:104D400070470000BFF34F8F024A1369DB03FCD4A6
:104D5000704700BF0020024008B5094B1B7873B9AB
:104D6000FFF7F0FF074B5A69002ABFBF064A9A6057
:104D700002F188329A601A6822F480621A6008BDD3
:104D8000503E0020002002402301674508B50B4B30
:104D90001B7893B9FFF7D6FF094B5A6942F00042DE
:104DA0005A611A6842F480521A601A6822F48052DA
:104DB0001A601A6842F480621A6008BD503E0020F2
:104DC000002002407F289ABF00F58030C0020020FA
:104DD000704700004FF4006070470000802070476B
:104DE0007F2808B50ED8FFF7EDFF0368013309D11E
:104DF00000F500630430834201D1012008BD026840
:104E00000132F7D00020F9E77F2810B504461FD8FB
:104E1000FFF798FFFFF7A0FF0E4BF3221A61022263
:104E20005A615A6942EAC0025A615A6942F48032B0
:104E30005A61FFF787FF4FF40061FFF7C3FF00F0EF
:104E40003BF9FFF7A3FF2046BDE81040FFF7C8BFBE
:104E5000002010BD0020024040EA02035B072DE95C
:104E6000F041144606D02E4B4FF461721A600020B8
:104E7000BDE8F0812B4B82189A420FD9284B40F2A3
:104E80008932F3E702680B689A420AD1031D1B6856
:104E90004A68934205D1083C08300831072CF1D804
:104EA00064B1FFF759FFFFF74DFF1F4E083101278F
:104EB0004FF00008012C03D8FFF768FF0120D7E767
:104EC0007761054651F8083C45F8043B51F8043C2D
:104ED0004360FFF737FF336943F001033361C6F8DE
:104EE0001480026851F8083C9A420DD00C4B40F2F5
:104EF000B1321A600D4B18600D4B1C600D4B083918
:104F00001960FFF743FFB2E72D6851F8042C954272
:104F100001F10803EAD1083C08301946CAE700BF8E
:104F20004C3E00200000040800200240483E0020C3
:104F3000443E0020403E0020084908B50B7828B1C7
:104F40001BB9FFF709FF01230B7008BD002BFCD034
:104F5000BDE808400870FFF719BF00BF503E0020B1
:104F600002484FF47F4100F0A9B800BF00010020C3
:104F700008461146FBF726BA0120FBF723BA0000CA
:104F80000846FBF741BA000038B5EFF311859DB92B
:104F9000EFF30584C4F30804302334B183F311889C
:104FA000FFF7B6FE85F3118838BD83F31188FFF74C
:104FB000AFFE84F3118838BDBDE83840FFF7A8BEC6
:104FC00038B5FFF7E1FF104C104AC00840EA4170C5
:104FD000A0FB025EC908A0FB040C1CEB05004FF00F
:104FE0000003A1FB04455B410019A1FB021043EB48
:104FF000050311EB0E0140F100005B1840F10000C9
:105000001B0943EA007038BDCFF753E3A59BC420CA
:1050100010B50244064BD2B2904200D110BD441CE0
:1050200000B253F8200041F8040BE0B2F4E700BFEF
:1050300050280040114B30B5D3F89040240409D4D7
:10504000D3F89040C3F89040D3F8904044F4004423
:10505000C3F890400A4C236843F4807323600244F1
:10506000084BD2B2904200D130BD441C00B251F87E
:10507000045B43F82050E0B2F4E700BF00100240A8
:10508000007000405028004007B5012201A900200F
:10509000FFF7BEFF019803B05DF804FB13B50446AB
:1050A000FFF7F2FFA04205D0012201A900200194E0
:1050B000FFF7C0FF02B010BD70470000704700004E
:1050C00070470000074B45F255521A6003225A60A0
:1050D00040F2FF729A604CF6CC421A60024B0122F9
:1050E0001A70704700300040513E0020034B1B787F
:1050F0001BB1034B4AF6AA221A607047513E0020AA
:1051000000300040054B1A6832B902F1804202F5C6
:105110000432D2F894201A60704700BF543E002039
:10512000024B4FF40002C3F8942070470010024075
:1051300008B5FFF7E7FF024B1868C0F3407008BDE1
:10514000543E002070470000704700007047000088
:10515000FEE700000A4B0B480B4A90420BD30B4B67
:10516000DA1C121AC11E22F00302994288BF0022E3
:105170000021FCF743BE53F8041B40F8041BECE786
:1051800010570008583E0020583E0020583E00208E
:1051900000F0C4B84FF08043586A70474FF0804326
:1051A000002258631A610222DA6070474FF0804390
:1051B0000022DA60704700004FF080435863704768
:1051C000FEE7000070B51B4B01630025044686B066
:1051D00085620E465860FEF7FDFF04F11003C4E936
:1051E00004334FF0FF33C4E90635C4E90044A56039
:1051F000E562FFF7CFFF2B460246C4E9082304F11E
:1052000034010D4A256580232046FFF7F3FB012377
:10521000E0600A4A0375009272680192B268CDE9B3
:105220000223074B6846CDE90435FFF70BFC06B0B7
:1052300070BD00BF383E0020E9550008EE5500085B
:10524000C1510008024AD36A0343D362704700BFCA
:10525000E03D0020274B2849DA6A42F0070210B4EB
:10526000DA62DA6A22F00702DA62DA6ADA6C42F0AB
:105270000702DA64DA6E42F00702DA664FF0904213
:10528000DB6E4FF0AA30002353604FF41924906076
:10529000D1604FF6FF71516113625462174C146074
:1052A000174CC2F80434C2F808444FF4A044C2F8C2
:1052B0000C444FF6FD74C2F814444FF0EE44C2F8AB
:1052C00020444AF20404C2F82434C2F80044C2F86C
:1052D0000438C2F80808C2F80C38C2F81418C2F82A
:1052E0002038C2F82438C2F800385DF8044B00F0CA
:1052F00055B800BF00100240000100240001802AC0
:10530000AAFAAAAA08B500F02BF9FFF74BFBBDE8F3
:105310000840FFF7F7BE0000704700000F4B9A6D82
:1053200042F001029A659A6F42F001029A670C4AB4
:105330009B6F936843F0010393604FF080434F22CB
:105340009A624FF0FF32DA6200229A615A63DA60A1
:105350005A6001225A611A60704700BF0010024073
:10536000002004E04FF0804208B51169D3680B407B
:10537000D9B2C9439B07116107D5302383F3118844
:10538000FFF736FB002383F3118808BD08B5FFF74C
:105390007FF8BDE8084000F0D7B800005B4B4FF045
:1053A000FF319A6A99629A6A00229A62986AD86A68
:1053B00060F00700D862D86A00F00700D862D86AA7
:1053C000186B1963186B1A63186B986B9963986B59
:1053D0009A63986BD86BD963D86BDA63D86B186C07
:1053E0001964196C1A641A6C494A4FF4E06111602F
:1053F0001A6E484942F001021A66D3F8802022F062
:105400000102C3F88020D3F880209A6D42F08052C8
:105410009A659A6F22F080529A679A6F4FF44072A1
:105420000A604A6912F48062FBD14A601A6822F06D
:10543000F00242F060021A601A6842F001021A603B
:105440001A689107FCD500229A609A6812F00C0243
:10545000FBD1D3F8901011F4407F1EBF4FF4803180
:10546000C3F89010C3F89020D3F8902042F01902AE
:10547000C3F89020D3F890209207FBD565221A60DC
:105480001A689007FCD500229A609A6812F00C0FF7
:10549000FBD16D221A60D3F8942022F4706242F49A
:1054A000C062C3F89420D3F8902022F00322C3F8FE
:1054B0009020194ADA601A6842F080721A601A68FD
:1054C0009101FCD5154A1A611A6842F080621A608F
:1054D0001A681201FCD500229A600D49104AC3F8DF
:1054E00088200A6822F0070242F004020A600A6873
:1054F00002F00702042AFAD19A6842F003029A6085
:105500009A6802F00C020C2AFAD17047001002408F
:105510000020024000700040012800010018100027
:105520005555013408B50348FEF72EFFBDE8084085
:10553000FEF774BE643B002008B5FFF713FFBDE81B
:105540000840FEF76BBE000008B507211C20FEF7DF
:10555000B3FFBDE808400C212520FEF7ADBF0000D9
:1055600008B5FFF713FF00F009F8FFF74FF9FFF751
:10557000D3FEBDE80840FFF70BBE000070470000F7
:105580000B4601461846FAF729BF00001211000029
:1055900012130000121000006F72672E61726475A2
:1055A00070696C6F742E3344522D4C3433312D415D
:1055B00053415541560053544D33324C343F3F0014
:1055C00040A2E4F1646891060041A3E5F2656992A6
:1055D00007004261642043414E496661636520696A
:1055E0006E6465782E006330006D61696E006964D9
:1055F0006C6500000000000000000000D1260008DB
:10560000A12E0008012E0008012700080D27000820
:1056100019290008D9260008E1260008DD2600081F
:1056200035280008E5260008B93100085531000882
:10563000F52600080928000880000000008000000E
:105640000000800000960000000000000000000044
:10565000000000000000000000000000000000004A
:10566000CD470008B9470008F5470008E1470008A2
:10567000ED470008D9470008C5470008B1470008B2
:1056800001480008E6550008D03B0020E03D00201E
:1056900024B3FF7F0100000004110020000000007F
:1056A0000000000068000000D000000000000000C2
:1056B00000000000000000000000000000000000EA
:1056C00000000000000000000000000000000000DA
:1056D00000000000000000000000000000000000CA
:1056E00000000000000000008D0400000000000029
:1056F0000000030000000000FE2A0100D2040000A8
:10570000FF000000643B002000000000B6550008C8
:00000001FF
